:1000000055EF05F00000000037EF05F0000000009C
:0A0010000000000000000000F3D71C
:10001C000FEE81F0EF50EFCF00F0009E00C0EFFF2D
:02002C001200C0
:0E002E00ACB202D00000FCD7D0C0ADFF120073
:10003C000FEE81F0EF50EFCF00F0009C00C0EFFF0F
:02004C001200A0
:06004E000000000012009A
:0A005400120E0D6E0D2EFED71200E5
:10005E00A69CCAC0A9FFA69EA680A8CF00F012003B
:10006E000B6A0A6A096A086A0E6A03340836045073
:10007E00085E0550D8A0053C095E0650D8A0063C87
:10008E000A5E0750D8A0073C0B5EE86AD8A0010EA6
:10009E000E5E0336070E0C6E0334083609360A362A
:1000AE000B360E36045003A012D0085E0550D8A0B1
:1000BE00053C095E0650D8A0063C0A5E0750D8A043
:1000CE00073C0B5EE86AD8A0010E0E5E11D0082622
:1000DE000550D8B0053C09260650D8B0063C0A2675
:1000EE000750D8B0073C0B26E86AD8B0010E0E2692
:1000FE0003360C2ED1D70234083609360A360B36A3
:10010E000E36045003A012D0085E0550D8A0053C50
:10011E00095E0650D8A0063C0A5E0750D8A0073CE0
:10012E000B5EE86AD8A0010E0E5E11D008260550AF
:10013E00D8B0053C09260650D8B0063C0A26075012
:10014E00D8B0073C0B26E86AD8B0010E0E26023650
:10015E00070E0C6E0234083609360A360B360E368A
:10016E00045002A012D0085E0550D8A0053C095ECE
:10017E000650D8A0063C0A5E0750D8A0073C0B5E7E
:10018E00E86AD8A0010E0E5E11D008260550D8B030
:10019E00053C09260650D8B0063C0A260750D8B0B2
:1001AE00073C0B26E86AD8B0010E0E2602360C2E3E
:1001BE00D1D70134083609360A360B360E360450BE
:1001CE0002A012D0085E0550D8A0053C095E06506C
:1001DE00D8A0063C0A5E0750D8A0073C0B5EE86A22
:1001EE00D8A0010E0E5E11D008260550D8B0053CE1
:1001FE0009260650D8B0063C0A260750D8B0073C50
:10020E000B26E86AD8B0010E0E260136070E0C6ECC
:10021E000134083609360A360B360E36045001A064
:10022E0012D0085E0550D8A0053C095E0650D8A035
:10023E00063C0A5E0750D8A0073C0B5EE86AD8A0C1
:10024E00010E0E5E11D008260550D8B0053C0926C9
:10025E000650D8B0063C0A260750D8B0073C0B26ED
:10026E00E86AD8B0010E0E2601360C2ED1D7003416
:10027E00083609360A360B360E36045001A012D057
:10028E00085E0550D8A0053C095E0650D8A0063C75
:10029E000A5E0750D8A0073C0B5EE86AD8A0010E94
:1002AE000E5E11D008260550D8B0053C0926065022
:1002BE00D8B0063C0A260750D8B0073C0B26E86A91
:1002CE00D8B0010E0E260036070E0C6E003408361E
:1002DE0009360A360B360E36045000A012D0085ED0
:1002EE000550D8A0053C095E0650D8A0063C0A5E13
:1002FE000750D8A0073C0B5EE86AD8A0010E0E5E30
:10030E0011D008260550D8B0053C09260650D8B0A5
:10031E00063C0A260750D8B0073C0B26E86AD8B030
:10032E00010E0E2600360C2ED1D700B00ED0045082
:10033E0008260550D8B0053C09260650D8B0063C14
:0C034E000A260750D8B0073C0B2612000E
:10035A00CAC002F0CBC003F002C000F003C001F033
:10036A00024A032A00C0E9FF01C0EAFFEE5201E097
:10037A00F3D70001CA51025C006ECB510358016EDB
:0A038A00010E005E000E015A120081
:100394000A0E0001D06F49DE0D0E0001D06F45DE5C
:0203A400120045
:1003A600086A096A100E0C6E0134083609360450C4
:1003B600085E0550D8A0053C095ED8B007D00450A9
:1003C60008260550D8B0053C0926D89000360136D7
:0603D6000C2EEAD7120014
:1003DC00010E0001CB6F000ECC6F800ECD6F000EA6
:1003EC00CE6FCD51CE1123E02CDE2BDE2ADE29DEA2
:1003FC000FDE939E26DE25DECD51CA15006E000E53
:10040C00CE15016E0050011002E0938C02D010DE6C
:10041C00939C17DE16DE938E709181BE04D070A172
:10042C0001D001D0FAD7CE33CD33CE9FDAD7CB6BF8
:10043C00CC6B07DE06DEECDD939E03DE02DE938CD6
:10044C0000DEFFDDFEDDFDDD938E709181BE04D0FC
:10045C0070A101D001D0FAD7CB6BCC6BF2DDF1DD02
:10046C0081AC01D0CB81EDDDECDDEBDDEADDE9DD4E
:10047C00E8DDE7DDE6DDE5DDE4DDE3DDE2DDE1DD64
:10048C00E0DDDFDDDEDDC4DD939ED2DD939CCBC0F1
:04049C0000F012005A
:1004A000CDDD939CD4DDD3DD938E0001709181BEB0
:1004B00004D070A101D001D0FAD7C9DDC8DDC7DDF5
:1004C000C6DDC5DDC4DDC3DDC2DD938CC0DDBFDDAF
:0204D000120018
:1004D200800E0001CC6F000ECD6FCE6BCF6BCC5176
:1004E200CD111BE0B3DDB2DD938CB0DDAFDD938EB9
:1004F200709181BE04D070A101D001D0FAD781AC35
:1005020004D0CC51CE13CD51CF13A0DD9FDD85DDBC
:10051200939ECD33CC33CD9FE2D7938C97DD96DD7E
:10052200CA51CB1102E089DD939C90DD8FDD938E61
:10053200709181BE04D070A101D001D0FAD786DDBE
:1005420085DD6BDD939E82DD81DD77DD939CCEC000
:0405520000F01200A3
:10055600938C7ADD79DD938E77DD76DD6CDD939C89
:0A05660073DD72DD58DD939E120074
:100570000001C06BC16BC26BC36BC00EC46F000EB9
:10058000C56F7651800F786F7F517827805178271B
:10059000E2DFD00ECA6F22DF78C0CAF01FDF80DF33
:1005A000DADFD10E0001CA6F19DF030EC425E16E38
:1005B000000EC521E26EE66A020EC425C66F000E6B
:1005C000C521C76F010ECA6F000ECB6F82DFC6C098
:1005D000E1FFC7C0E2FF00C0E6FF010EC425C66F01
:1005E000000EC521C76F010ECA6F000ECB6F71DF01
:1005F000C6C0E1FFC7C0E2FF00C0E6FFC4C0C6F04E
:10060000C5C0C7F0010ECA6F000ECB6F62DFC6C057
:10061000E1FFC7C0E2FF00C0E6FFCA6BCB6B59DF4A
:100620003FDFC0C000F0C1C001F0C2C002F0C3C0D3
:0406300003F01200C1
:100634004EC0CAF04FC0CBF08EDE00C0C1F0C06B1C
:10064400C0514E24E96E000EC0BFFF0E4F20EA6E6B
:10065400EECFD0F0EADC0001C02B800EC019006E92
:10066400800EC119005CECE319D029D028D02C0EDF
:10067400D06FDBDC24D0090E0001D06FD6DC1FD094
:100684000D0E0001D06FD1DC0A0E0001D06FCDDC5D
:1006940016D02A0E0001D06FC8DC11D000017751AA
:1006A400000AE3E07751010AE1E07751030ADFE051
:1006B4007751050AE0E07751070AE2E0EAD7120031
:1006C400220E0C6E086A096A0A6A0B6A0C06D8B410
:1006D4001FD0D8900B320A32093208320332023268
:1006E40001320032D8A0F2D70C06D8B409D0045095
:1006F40008260550092206500A2207500B22EAD781
:10070400045008260550092206500A2207500B22DD
:020714001200D1
:100716002E0E0001716F000E726FD00E736F000EF9
:10072600746FBC0E646F070E656F000E666F000E69
:10073600676FCE0E6C6F070E6D6F000E6E6F000E3C
:100746006F6FFF0E686FFF0E696F000E6A6F000E07
:100756006B6FAC8A900EAB6E948E949C9EAA03D05F
:08076600AECF00F0FBD712003A
:10076E00C0C004F0C1C005F004C002F005C003F023
:10077E00044A052AC2C000F0C3C001F00001C24BFA
:10078E00C32B00C0E9FF01C0EAFF02C0E1FF03C0B6
:10079E00E2FFEECFE6FF02C0E9FF03C0EAFFEE5232
:0E07AE0001E0E2D7C0C000F0C1C001F01200AF
:1007BC00AECF75F0ABA202D0AB98AB8875C000F091
:0207CC00120019
:0A07CE00000E9EBA010E006E12002C
:1007D8000001C66BC76B000EC75D02E10A0EC65D5D
:1007E8000BE2C651C425E16EC751C521E26E200E49
:1007F800E66EC64BC72BEFD7C651C425E16EC7516D
:10080800C521E26EE66A010EC65F000EC75BC651DF
:10081800C425C86FC751C521C96F0A0E046E000EE2
:10082800056E066E076EC0C000F0C1C001F0C2C000
:1008380002F0C3C003F017DC08C000F009C001F0E3
:100848000AC002F00BC003F0300E0026C8C0E1FF5A
:10085800C9C0E2FF00C0E6FF0A0E046E000E056E76
:10086800066E076EC0C000F0C1C001F0C2C002F041
:10087800C3C003F037EC00F000C0C0F001C0C1F005
:1008880002C0C2F003C0C3F0000E046E031808E1F2
:100898000450021805E10450011802E10050000A52
:1008A80001E105D0010EC65F000EC75BB0D712008C
:1008B8006DDD100E0001C26F000EC36FC2C0CAF01A
:1008C8002FEC00F000C0C0F0000EC16F000EC1197F
:1008D80002E1000EC01901E119D0110E0C6E3A0E9A
:1008E8000D6E0D2EFED70C2EFCD70000C0C0D0F028
:1008F80017EC00F00001C24BC32B800EC319006E29
:10090800800E005C02E1500EC25DD8E33FDD1200AC
:10091800C0C004F0C1C005F004C0E9FF05C0EAFF8B
:10092800EE5203E0044A052AF7D704C002F005C0D6
:1009380003F0044A052AC2C000F0C3C001F0000158
:10094800C24BC32B00C0E9FF01C0EAFF02C0E1FFB0
:1009580003C0E2FFEECFE6FF02C0E9FF03C0EAFFF3
:10096800EE5201E0E2D7C0C000F0C1C001F01200B1
:10097800C26AC00EC212C18CC18EC0C000F000365F
:10098800009000360090003600900050C212C280DD
:100998002AEC00F0C284C2A401D0FDD7C4CF01F074
:0E09A800006AC3500012000E0112C29012002D
:1009B600938E938C0001709181BE04D070A101D0FA
:0609C60001D0FAD7120077
:1009CC000001C46B050EC45D0AE2C451C225E16E80
:1009DC00000EC321E26E200EE66EC42BF3D7C45179
:1009EC00C225E16E000EC321E26EE66AC407C45153
:1009FC00C225C56F000EC321C66F0A0E046E000E11
:100A0C00056EC0C000F0C1C001F0C7DC08C000F02A
:100A1C0009C001F0300E0026C5C0E1FFC6C0E2FFE0
:100A2C0000C0E6FF0A0E046E000E056EC0C000F09A
:100A3C00C1C001F0B2DC00C0C0F001C0C1F0000EBA
:100A4C00011802E1000E001801E102D0C407CFD753
:020A5C00120086
:100A5E000900F5CFE6FF0006FBE10106F9E1120001
:100A6E0000C015F09EA017D000017D4B7E2B0B0E03
:100A7E00CF6EDB0ECE6E9E90000E006E7E51005C31
:100A8E0002E17D51050806E2794B7A2B7D6B7E6B78
:0C0A9E00010E526E9E9015C000F0110079
:100AAA0019EC08F0FC0EF66E0F0EF76E000EF86EDB
:100ABA00820EE16E000EE26E360E006E010E016EBF
:100ACA00C9DF6F6A6E6AFC0E936EF18EFF0E8A6E34
:100ADA00FF0E806EFF0E926E810EC26E890EC16E7F
:100AEA00946A010ED56E0A0EAF6EAC840FDE6ADE12
:100AFA000050010A03E15DDE00C081F00001816B54
:100B0A00030E776F42DC4EC0C0F04FC0C1F0820EB8
:100B1A000001C26F000EC36F25DE00C04EF001C097
:100B2A004FF083DD32DC0001BC6BBD6B000EBD5D96
:100B3A0002E10F0EBC5D18E2BCC0CAF02FEC00F057
:100B4A0000C0BAF0000EBB6FA30E0C6E550E0D6EF0
:100B5A000D2EFED70C2EFCD7BAC0D0F017EC00F041
:100B6A000001BC4BBD2BE2D710DC030E0001776FEE
:100B7A007B6B7C6B816B7D6B7E6B796B7A6BB86BF5
:100B8A00B96B7B6B7C6B000E7C5D02E1040E7B5DB6
:100B9A0054E27BC000F07CC001F0003600900136C0
:100BAA00003600900136530E0024BE6F000E01205D
:100BBA00BF6F7BC000F07CC001F0000E026E036EB6
:100BCA00A00E046E8C0E056E000E066E076E75DDA5
:100BDA000D0E0026020E0122000E02220322BEC0C2
:100BEA00E1FFBFC0E2FF00C0E6FF01C0E6FF02C0AE
:100BFA00E6FF03C0E6FF7BC000F07CC001F00036D0
:100C0A0000900136003600900136530E0024E96E3A
:100C1A00000E0120EA6EEECFC0F0EECFC1F0EECFAB
:100C2A00C2F0EECFC3F04EC0C4F04FC0C5F0CFDD66
:100C3A00FCDC00017B4B7C2BA6D7CAEC01F0B6DEAC
:100C4A00300ECD6ECD80DB0ECF6E0B0ECE6E9E902B
:100C5A00F28C9D80F28E030E0001776FB86BB96B30
:100C6A004EC0C0F04FC0C1F0A00EC26F000EC36FDD
:100C7A0079DD00C04EF001C04FF0D7DC0001766B81
:100C8A000C0E7F6F806B8C0E786F8C0EC06F000E0F
:100C9A00C16F4EC0C2F04FC0C3F093DEBA6BBB6BDC
:100CAA00000EBB5D02E1040EBA5D16E2BA514E2493
:100CBA00E96EBB514F20EA6EEECF01F00150200AD7
:100CCA0008E1BA514E24E16EBB514F20E26E300E5C
:100CDA00E66EBA4BBB2BE4D7A8DCCAEC01F0020ED5
:100CEA000001636F816B7B6B7C6BE1DD6BDD005018
:100CFA00010A37E15EDD00C081F019D0000163719D
:100D0A0030D063732ED063752CD0030E805D01E260
:100D1A00802B27D08051000801E2800722D0C7DD4E
:100D2A0020D0CAEC01F0CAEC01F01BD01AD00001A5
:100D3A008151310AE3E08151320AE3E08151330AF9
:100D4A00E2E081512B0AE1E081512D0AE3E0815171
:100D5A00450AE5E08151650AE2E081511B0AE1E0BA
:100D6A00E5D70001B84BB92B030E776F090ED06F88
:100D7A0017EC00F0000163A142D04EC0C0F04FC092
:100D8A00C1F0AF0EC26F000EC36FECDC00C04EF0B4
:100D9A0001C04FF0B8C0C0F0B9C0C1F01AC0C2F06B
:100DAA001BC0C3F00EDEBA6BBB6B000EBB5D02E16B
:100DBA00050EBA5D16E2BA511A24E96EBB511B2020
:100DCA00EA6EEECF01F00150200A08E1BA511A2466
:100DDA00E16EBB511B20E26E300EE66EBA4BBB2BA6
:100DEA00E4D74EC0C0F04FC0C1F01AC0C2F01BC059
:100DFA00C3F08DDD00C04EF001C04FF016DC0001DB
:100E0A0063A33BD0BA6BBB6B000EBB5D02E1050E60
:100E1A00BA5D33E24EC0C0F04FC0C1F0B30EC26F2C
:100E2A00000EC36F9FDC020E4E24E16E000E4F20AF
:100E3A00E26E300EBA25006E00C0E6FFBAC0C0F0FE
:100E4A0096DD00C050F001C051F000C0C0F001C0F2
:100E5A00C1F01AC0C2F01BC0C3F0B3DD4EC0C0F06F
:100E6A004FC0C1F01AC0C2F01BC0C3F050DD1AEC6B
:100E7A0003F00001BA4BBB2BC7D77B6B7C6B030E0D
:100E8A00776F0CD0200E766F22D0400E766F1FD06F
:100E9A00600E766F1CD0766B1AD019D0000E7C19B2
:100EAA0002E1000E7B19EEE0000E7C1902E1010E50
:100EBA007B19EBE0000E7C1902E1020E7B19E8E0D7
:100ECA00000E7C1902E1030E7B19E5E0E6D763A563
:100EDA0019D07BC000F07CC001F0003600900136CA
:100EEA00003600900136530E0024E96E000E0120F0
:100EFA00EA6EEECF16F0EECF17F0EECF18F0EECF87
:100F0A0019F00AD0B8EC02F000C016F001C017F0D0
:100F1A0002C018F003C019F016C0C0F017C0C1F023
:100F2A0018C0C2F019C0C3F04EC0C4F04FC0C5F01B
:100F3A004EDC1AEC03F0040E0B6E2C0E0C6EAB0E8C
:100F4A000D6E0D2EFED70C2EFCD70B2EFAD70000F5
:100F5A00000000017B4B7C2B000E7C5D02E1040E3D
:100F6A007B5D8FE3090ED06F17EC00F080C0C0F0F4
:100F7A00000E0001C16F4EC0C2F04FC0C3F021DDA8
:100F8A001AEC03F0CAEC01F0F2BE0FD0020E0B6E9F
:100F9A00450E0C6EA90E0D6E0D2EFED70C2EFCD72B
:100FAA000B2EFAD70000000004D05250000AFDE0D0
:080FBA00526A8A729BD6FFD730
:1010320010EE16F03A0E006E010E016EC20EF66E42
:0E1042000F0EF76E000EF86E2FEC05F0120088
:040FC200000000002B
:020FC6001C000D
:100FC80031323334353637383930313233343536D7
:010FD8000018
:100FD90031323334353637383930313233343536C6
:100FE90037383930313233343536373839303132B0
:010FF90000F7
:020FFA002D00C8
:100FFC00204D435033343234204144432031382087
:0E100C00626974732031332F30392F31300078
:0F101A00436F6E666967204144433138623D0081
:041029004E623D00D6
:05102D004348303D00C6
:020000040030CA
:0D00010022050EFFFF80FF0FC00FE00F4033
:0200000400F00A
:100000007061756C666A756A6F40667265652E0010
:1000100034434820414443313062697473200909F4
:1000200020436F6E7369676E65733A202031366DB9
:1000300056202036346D56202020203132386D561F
:100040002020203230306D562020204741494E007C
:10005000FFFFFFFFFFFFFFFFFFFFFFFFFFFFFFFFB0
:10006000FFFFFFFFFFFFFFFFFFFFFFFFFFFFFFFFA0
:10007000FFFFFFFFFFFFFFFFFFFFFFFFFFFFFFFF90
:10008000FFFFFFFFFFFFFFFFFFFFFFFFFFFFFFFF80
:10009000FFFFFFFFFFFFFFFFFFFFFFFFFFFFFFFF70
:1000A000FFFFFFFFFFFFFFFFFFFFFFFFFFFFFFFF60
:1000B000FFFFFFFFFFFFFFFFFFFFFFFFFFFFFFFF50
:1000C000FFFFFFFFFFFFFFFFFFFFFFFFFFFFFFFF40
:1000D000FFFFFFFFFFFFFFFFFFFFFFFFFFFFFFFF30
:1000E000FFFFFFFFFFFFFFFFFFFFFFFFFFFFFFFF20
:1000F000FFFFFFFFFFFFFFFFFFFFFFFFFFFFFFFF10
:00000001FF
